:100000000C943E020C9476020C9476020C947602C8
:100010000C9476020C9476020C9476020C94760280
:100020000C9476020C9476020C94D2250C94A4269F
:100030000C94B1200C9476020C9476020C94760207
:100040000C9476020C9476020C9476020C94760250
:100050000C9476020C9439210C9476020C9476025E
:100060000C9476020C9476020C9476020C94760230
:100070000C9476020C9476020C9476020C94760220
:100080000C9476020C9476020C9476020C94760210
:100090000C9476020C9476020C9476020C94760200
:1000A0000C9476020C9476020C947602380538058E
:1000B00064056405CC05EA0502070207F5058E060E
:1000C0009F069F0611273827302838273028842795
:1000D000A7273028FE270D284C0052002800C45CBA
:1000E000500051004F000151C65CCA5CC85C010061
:1000F000C75CCB5CC95C010000047F3F1F64321405
:10010000643214783C1E1E140A0522232526282951
:100110002A2C2D2F3032333536383A3B3D3E404283
:10012000434547494A4C4E5051535557595A5C5EC6
:100130006062646668696B6D6F71737577797B7DDA
:100140007F81838587898A8C8E90929496989A9CD9
:100150009E9FA1A3A5A7A8AAACAEAFB1B3B4B6B8F1
:10016000B9BBBCBEBFC1C2C3C5C6C7C9CACBCCCD53
:10017000CED0D1D2D2D3D4D5D6D7D7D8D9D9DADA2E
:10018000DBDBDBDCDCDCDCDCDDDDDDDDDCDCDCDCAE
:10019000DCDBDBDBDADAD9D9D8D7D7D6D5D4D3D2E2
:1001A000D2D1D0CECDCCCBCAC9C7C6C5C3C2C1BFC0
:1001B000BEBCBBB9B8B6B4B3B1AFAEACAAA8A7A524
:1001C000A3A19F9E9C9A98969492908E8C8A8987E0
:1001D0008583817F7D7B79777573716F6D6B6968BE
:1001E000666462605E5C5A5957555351504E4C4A92
:1001F0004947454342403E3D3B3A3836353332303D
:100200002F2D2C2A292826252322FFAA7F5540009E
:1002100001010101010101010102020202020202C7
:10022000020203030303030303030404040404049A
:100230000405050505050606060606070707070760
:1002400008080808090909090A0A0A0B0B0B0C0C13
:100250000C0D0D0D0E0E0E0F0F0F101011111112AF
:100260001213131414151516161717181819191A2E
:100270001A1B1B1C1D1D1E1E1F2020212222232491
:1002800024252626272829292A2B2C2D2D2E2F30D0
:10029000313232333435363738393A3B3C3D3E3FE4
:1002A000404142434445464748494A4C4D4E4F50D1
:1002B000515354555658595A5B5D5E5F616264658F
:1002C0006668696B6C6D6F7072737577787A7B7D19
:1002D0007E8082838587888A8C8E8F91939596986D
:1002E0009A9C9EA0A2A3A5A7A9ABADAFB1B3B5B789
:1002F000BABCBEC0C2C4C6C9CBCDCFD1D4D6D8DB60
:10030000DDDFE2E4E7E9EBEEF0F3F5F8FAFDFF0AF2
:100310000353004F0041005000000018034B0069D8
:10032000006E0067006C0079002D004B00650079BD
:1003300000730000000403090409023B00020100ED
:10034000A0FA0904000001030101000921110100C4
:100350000122400007058103080001090401000192
:100360000300000009211101000122B600070582E7
:10037000032000011201000200000008EDFE03004E
:1003800004000102000105010902A1018502090121
:10039000A100050919012908150025019508750115
:1003A00081020501093009311581257F9502750803
:1003B000810609381581257F950175088106050C90
:1003C0000A38021581257F950175088106C0C00590
:1003D000010980A101850319012AB700150126B77B
:1003E00000950175108100C0050C0901A10185046B
:1003F00019012AA002150126A0029501751081009D
:10040000C005010906A1018506050719E029E715C0
:100410000025019508750181020507190029EF15CE
:1004200000250195F075018102050819012905953E
:100430000575019102950175039101C00501090639
:10044000A101050719E029E71500250195087501A7
:1004500081029501750881010507190029FF150022
:1004600026FF0095067508810005081901290595E4
:100470000575019102950175039101C011241FBEFC
:10048000CFEFDAE0DEBFCDBF04B603FE18C0809127
:10049000DB029091DC02A091DD02B091DE02873098
:1004A000904BA740B04B59F41092DB021092DC0243
:1004B0001092DD021092DE02E0E0F8E3099511E00F
:1004C000A0E0B1E0E6ECF2E502C005900D92AA3C96
:1004D000B107D9F722E0AAECB1E001C01D92AB3D13
:1004E000B207E1F70E94DC120C9461290C94000021
:1004F000811107C0662311F08BEF01C08CEF0E94C1
:10050000E60481E0089581E0089581E008950C9467
:10051000850208950C9489021F93CF93DF9300D036
:1005200000D01F92CDB7DEB749835A836B833091D9
:10053000CD0189819A81311114C0662359F022239B
:1005400049F00E943D09182F682F89819A810E94E5
:10055000E80803C00E941209182F69817A81812F4F
:1005600004C00E943D0969817A810F900F900F901D
:100570000F900F90DF91CF911F910C947C10FC0194
:10058000262F408151816281738184810C948C0279
:1005900081E00895CF93DF93EC0160E00E94BF02F9
:1005A000BE01DF91CF910C948A020C94BF110C9480
:1005B000BB1108950E9492070E94D9022FEF84E395
:1005C0009CE0215080409040E1F700C000000C9476
:1005D0005F210F931F93CF93DF938C0161E00E9403
:1005E000BF02EC01B8010E948702882309F444C0CD
:1005F000B801CE010E94FB1E8823F1F1B801CE01A3
:100600000E949E1C8823C1F1B801CE010E94571E92
:10061000882391F1B801CE010E94A41B882361F1C7
:10062000F8018281882309F1CB358DE5D807C1F027
:1006300050F4C115FCE5DF0781F0CF3DDC45A9F49E
:100640000E94740E19C0CC35EDE5DE0761F0CD35A2
:10065000DD4559F40E94B70D08C00E94DA020CC0B3
:100660000E94C00D02C00E94C30DC801DF91CF914E
:100670001F910F910C94830280E0DF91CF911F9125
:100680000F9108950E9492200C945B030E945E03D8
:100690000C94982008950C944A0381E008950C94DA
:1006A0004D030895CF93C82F0E944B038C2F0E94B7
:1006B0004F03CF91089580E00C9452030E94571F7E
:1006C0000C9452030E94571F9091CC01891721F07E
:1006D0008093CC010C9452030895CF93DF93CDB750
:1006E000DEB72B970FB6F894DEBF0FBECDBF4F839A
:1006F000588769877A878B8761110E94030D9E0155
:100700002F5F3F4F86E0F90111928A95E9F785E066
:10071000FE013796D90101900D928A95E1F7898102
:100720009A814C815D81452B31F09F3F31F491E0FE
:100730008F3F19F403C091E001C090E090FF09C021
:1007400049815A816B817C818D819E810E94240C1C
:1007500005C0C9010E94C8028111F2CF2B960FB6C5
:10076000F894DEBF0FBECDBFDF91CF910895FC019D
:10077000808191810E947F090895CF93882309F495
:10078000A4C0C82F8238C1F40E94571F81FD9DC0AC
:1007900069E380910201909103010E944D200E9423
:1007A000250D2FEF81EE94E0215080409040E1F73D
:1007B00000C0000069E319C0833801F50E94571F8B
:1007C00080FD83C063E580910201909103010E9446
:1007D0004D200E94250D2FEF81EE94E021508040A6
:1007E0009040E1F700C0000063E580910201909124
:1007F00003010E945820CF910C94250D8438C1F438
:100800000E94571F82FD61C067E4809102019091B0
:1008100003010E944D200E94250D2FEF81EE94E0F0
:10082000215080409040E1F700C0000067E4DDCF38
:100830008CEF8C0F813AD0F46C2F80910201909153
:1008400003010E94CD1F882349F06C2F8091020183
:10085000909103010E9458200E94250D6C2F8091D9
:100860000201909103010E944D20C5CF80E28C0FC0
:10087000883048F4C77081E001C0880FCA95EAF754
:100880000E94E60CB8CFEBE5EC0FE33040F4F0E06B
:10089000E65AFE4F808190E0CF910C948B1FE8E5E3
:1008A000EC0FE73150F4F0E0EE0FFF1FE45DFE4F78
:1008B00080819181CF910C94A11FCD3E30F08C2F7F
:1008C0000E946113CF910C943314CF910895882323
:1008D00009F464C0823879F40E94571F81FF5EC01A
:1008E00069E380910201909103010E944D200E94D2
:1008F000250D69E310C08338B1F40E94571F80FFB3
:100900004DC063E580910201909103010E944D204A
:100910000E94250D63E580910201909103010E94E0
:1009200058200C94250D843879F40E94571F82FFBB
:1009300035C067E480910201909103010E944D202F
:100940000E94250D67E4E7CF9CEF980F913A10F4D1
:10095000682FE1CF90E2980F983050F4877091E0C3
:1009600001C0990F8A95EAF7892F0E94EC0CD9CF24
:100970009BE5980F933020F480E090E00C948B1F5F
:1009800098E5980F973120F480E090E00C94A11F37
:100990008D3E20F00E94BC130C94331408951F93D5
:1009A000CF93DF93182FEB010E94BD03209741F0F6
:1009B0008FE99FE00197F1F700C000002197F6CF83
:1009C000812FDF91CF911F910C946704893319F027
:1009D00060E070E002C060E570E00C94CF04882312
:1009E00021F00E94E60C0C94250D0895882321F037
:1009F0000E94EC0C0C94250D0895CF92DF92EF929B
:100A0000FF920F931F93CF93DF937C01D62FC72FB5
:100A1000FC011281058102950F700E94DC0C882375
:100A2000B9F01123A9F08C2F807F803421F080E26F
:100A30008D0F883068F08091B70282FD09C082E096
:100A40000E94850D0E94DC0C91E0D82ED92601C0B1
:100A5000D12CCC2EC2948FE0C8228C2D90E08C300B
:100A6000910508F0CFC1FC01EA5AFF4F0C94BC2855
:100A70008C2F807FCF70882311F0C295C07F112307
:100A800099F0CC2309F4AAC180E28D0F883010F0D0
:100A9000D11104C08C2F0E94E60C03C08C2F0E9441
:100AA000F60C0E94250D9AC18D2F0E946704CC235D
:100AB00009F4A8C180E28D0F883038F1DD2329F1D7
:100AC0008C2F0E94FC0C24C08C2F807FCF70803232
:100AD00011F0C295C07FDD2319F0D130A1F13DC0E6
:100AE0008091B70282FF17C0112349F0CC2329F06F
:100AF0008C2F0E94E60C0E94250D80E070C180E0E2
:100B00000E946704CC2309F47DC18C2F0E94EC0C59
:100B10000E94250D77C1112371F0002341F00130AF
:100B200031F40E94060D8C2B0E940E0D6BC10E94A9
:100B3000060D8C2B1DC0002319F0013009F462C191
:100B40000E941B0D25C0112321F0063008F05AC168
:100B50000EC0053008F056C11BC0112361F0002300
:100B600031F0F701858180FF39C18F7085838C2F2B
:100B70000E94EF0447C1002359F0D93309F03FC167
:100B8000FFEF07EE13E0F15000401040E1F735C1F0
:100B90008C2F0E94F60436C18C2F86958695837023
:100BA00019F0813061F02EC1112321F08D2F9C2F7F
:100BB000937002C080E090E00E948B1F2BC1112334
:100BC00021F08D2F9C2F937002C080E090E00E9456
:100BD000A11F20C18D2F112319F00E94611302C0A3
:100BE0000E94BC130E94331415C18C2F837009F02E
:100BF00047C011110BC12D2F229526952770220F6A
:100C0000220F6D2F6F70862F90E0A0E0B0E0022ED3
:100C100004C0880F991FAA1FBB1F0A94D2F7D4FFE4
:100C200010C04FE050E060E070E004C0440F551F7A
:100C3000661F771F2A95D2F740955095609570955D
:100C400003C040E050E0BA01C695C695C3708A0162
:100C50009B01082B192B2A2B3B2BC901B801C23051
:100C600049F058F4C13019F00E94FE07CFC00E942D
:100C7000EC07CCC00E941008C9C00E94EA07C6C099
:100C8000112319F08C2F817001C08695882309F4F7
:100C9000BDC02D2F229526952770220F220F6D2F74
:100CA0006F70862F90E0A0E0B0E0022E04C0880FA5
:100CB000991FAA1FBB1F0A94D2F7D4FF10C04FE0A0
:100CC00050E060E070E004C0440F551F661F771FBE
:100CD0002A95D2F7409550956095709503C040E0F5
:100CE00050E0BA01C695C695C3708A019B01082BD6
:100CF000192B2A2B3B2BC901B801C23049F058F4FB
:100D0000C13019F00E94C30881C00E94B1087EC0A2
:100D10000E94D5087BC00E94240878C0CF701123A0
:100D200039F08C2F0E944A088D2F0E94EF046EC06C
:100D30008D2F0E94F6048C2F0E946B0867C0D23F53
:100D400021F128F4D03F41F0D13FC1F043C0D33F5F
:100D500019F1D43F79F03EC0112341F0053008F07D
:100D600051C08C2F8F710E9490084CC0063008F043
:100D700049C0F7CF8091B70282FF18C0112339F024
:100D80008C2F8F710E944A083DC01123C9F38C2F0C
:100D90008F710E946B0836C0112329F08C2F8F7140
:100DA0000E9435082FC00E9430082CC0112349F042
:100DB000CF718C2F0E944A0863E08C2F0E946A0D2D
:100DC00021C081E00E94850D0230E0F082E00E94A7
:100DD000850D18C0112331F0002391F28D2F0E9450
:100DE000BD0310C0002399F2D93349F41FEF27EE59
:100DF00033E0115020403040E1F700C000008D2F5B
:100E00000E94670488EF8C0D843020F40E94571FE5
:100E10000E945203DD20C9F00E94D80C80FD15C04D
:100E2000F70112820E94D20C0E944A08C7010E9458
:100E300046070E94D20CDF91CF911F910F91FF9036
:100E4000EF90DF90CF900C946B08DF91CF911F91C2
:100E50000F91FF90EF90DF90CF9008950F931F9325
:100E6000CF93DF93EC01688179818A810E948A099E
:100E70008C010E94E7080E94D807B801CE010E94A9
:100E8000FD04DF91CF911F910F910895CF93DF93D0
:100E9000EC01988189812B813C81232B31F08F3F9C
:100EA00031F481E09F3F19F403C081E001C080E08C
:100EB00080FD1DC0CE010E94E902811110C00E9478
:100EC000DC0C8823A1F08A81882389F08091B70205
:100ED00082FD0DC082E0DF91CF910C94850DCE0193
:100EE0000E942E07CE01DF91CF910C94CA02DF91B0
:100EF000CF91089580E090E00E948B1F80E090E009
:100F00000E94A11F0E94030D0E94250D0E946415DE
:100F10000C94331480910201909103010E9463208C
:100F20000C947A070E94F30C0C948A0792959F7098
:100F3000963079F010F4925001C09A50923068F4D3
:100F4000803F69F018F4883E40F409C0843F29F4DA
:100F500006C0883E20F0813F11F080E0089581E0D6
:100F60000895FC01808191810E947F090E9496076B
:100F70000895CF93DF9300D000D01F92CDB7DEB796
:100F80000F900F900F900F900F90DF91CF910895D9
:100F9000CF93DF9300D000D000D0CDB7DEB7269638
:100FA0000FB6F894DEBF0FBECDBFDF91CF9108958D
:100FB000089508950C94D9070C94DA070E94DC0771
:100FC0006093D7017093D8018093D9019093DA018F
:100FD0000C947A070C94DE070F931F930091D701AE
:100FE0001091D8012091D9013091DA01602B712B39
:100FF000822B932B1F910F910C94DE070F931F935D
:101000000091D7011091D8012091D9013091DA01D6
:1010100060237123822393231F910F910C94DE0789
:101020000F931F930091D7011091D8012091D901FE
:101030003091DA0160277127822793271F910F9142
:101040000C94DE070C94D9070E9422086093D30108
:101050007093D4018093D5019093D6010C947A07B4
:1010600060E070E0CB010C9424080F931F9341E0E3
:1010700050E060E070E08A019B0104C0000F111F86
:10108000221F331F8A95D2F7C901B8011F910F9112
:101090000C9424080F931F9341E050E060E070E04F
:1010A00004C0440F551F661F771F8A95D2F78091A1
:1010B000D3019091D401A091D501B091D6018A01BC
:1010C0009B01082B192B2A2B3B2BC901B8011F911F
:1010D0000F910C9424080F931F9341E050E060E0BF
:1010E00070E004C0440F551F661F771F8A95D2F722
:1010F00040955095609570958091D3019091D40161
:10110000A091D501B091D6018A019B010823192332
:101110002A233B23C901B8011F910F910C94240885
:101120000F931F9341E050E060E070E004C0440F73
:10113000551F661F771F8A95D2F78091D301909132
:10114000D401A091D501B091D6018A019B01082755
:1011500019272A273B27C901B8011F910F910C9429
:1011600024080F931F930091D3011091D401209173
:10117000D5013091D601602B712B822B932B1F91BF
:101180000F910C9424080F931F930091D301109199
:10119000D4012091D5013091D6016023712382239F
:1011A00093231F910F910C9424080F931F93009188
:1011B000D3011091D4012091D5013091D60160273F
:1011C0007127822793271F910F910C94240808956B
:1011D000990F990F890FE82FE695E695E6958770A8
:1011E00051E001C0550F8A95EAF785E0E89FF001CC
:1011F0001124E253FE4F20E030E070E04081CB014B
:10120000022E02C0969587950A94E2F78170819527
:1012100084278523842781932F5F3F4F2530310515
:1012200069F70895990F990F890F682F669566954C
:101230006695982F977085E0689FB001112440E073
:1012400050E080E0FB01E40FF51FE253FE4F2081E8
:1012500030E0092E02C0369527950A94E2F72170F6
:101260003327042E01C0220F0A94EAF7822B4F5F26
:101270005F4F4530510531F70895BF92CF92DF920D
:10128000EF92FF920F931F93CF93DF938C01C09047
:10129000D301D090D401E090D501F090D601809197
:1012A000D7019091D801A091D901B091DA01C82A53
:1012B000D92AEA2AFB2ACFE1D0E0D701C6010C2EB9
:1012C00004C0B695A795979587950A94D2F780FDA7
:1012D00004C0219790F7B12C07C0BC2EB8018C2F09
:1012E0000E948F100197A9F38B2DDF91CF911F9151
:1012F0000F91FF90EF90DF90CF90BF900895CF9324
:10130000DF93EC010E943D09BE010E948F10DF9126
:10131000CF9108951F93CF93DF93EB019091CD016F
:10132000992321F0CB010E947F0913C0882349F043
:10133000CB010E943D09182F682FCE010E94E808BA
:1013400004C0CB010E941209182FBE01812F0E94F8
:101350008F10DF91CF911F9108951F93CF93DF934B
:10136000C091DB0116E08091DC01C81799F0D0E054
:101370001C9FF0011D9FF00D1124E352FE4F408190
:10138000518162817381848195810E94C807219671
:10139000C770E9CFDF91CF911F91089540910D0261
:1013A00050910E0260910F02709110028091110213
:1013B000909112020C94C807EF92FF920F931F9323
:1013C000CF93DF938091120282958F7009F065C0F0
:1013D00080910F02882309F460C08091DB01F090B6
:1013E000DC0110910D0200910E02609110027091CB
:1013F000110291E01F3F09F090E0C0910001D091EF
:101400000101292F96E0E92E8F1509F446C06115D8
:10141000710521F00F3F21F030E003C031E001C041
:10142000322F90E030FD36C0E89EF001E99EF00DCD
:101430001124DF01A352BE4F11963C911197301336
:1014400029C03C91311326C012963C91129731115C
:1014500021C013964D915C911497461B570B4C1766
:101460005D07C0F4809112028F7080618093120238
:10147000EE51FE4F80818F70806180838DE092E01D
:101480000E944607DF91CF911F910F91FF90EF903F
:101490000C94AD0901968770B7CFDF91CF911F9162
:1014A0000F91FF90EF9008959F92AF92BF92CF92CD
:1014B000DF92EF92FF920F931F93CF93DF93CDB7FD
:1014C000DEB761970FB6F894DEBF0FBECDBF8C01BB
:1014D00085E0F801DE011D9601900D928A95E1F7F5
:1014E000D8011296EC9090910D02E0910E0220919D
:1014F0001002309111022115310531F0EF3F31F426
:1015000081E09F3F19F403C081E001C080E0B82F63
:10151000B1709B2E80FD47C1D8014C9111965C9112
:1015200011971396AD90BC9014978DE0C82E82E071
:10153000D82EF0900F02B501621B730B20910001B1
:1015400030910101FF2009F4D9C080911202621785
:10155000730708F095C0282F207F09F052C05E1352
:1015600013C0491311C0FE2CE1100EC08F708061B2
:10157000809312020E94CE09C6010E944607809104
:101580001202F80185834DC1AB2831F05F3F31F481
:1015900081E04F3F19F403C081E001C080E080FD8D
:1015A00003C081E08E2502C080E090E0F82FF1704A
:1015B000FF2E80FF1CC08091DB012091DC0136E012
:1015C000821709F40BC190E0389FF001399FF00DAC
:1015D0001124E352FE4F6181561306C06081461309
:1015E00003C06281E61203C001968770E9CFFE2C2A
:1015F000EE2009F416C180911202816080931202DC
:1016000054C05E1306C0491304C0E11002C0F801C3
:1016100099C0C8010E94B107882361F1EE2051F101
:1016200020911202822F82958F7090E0029774F0C1
:1016300080910D0290910E0298878F831986BB8648
:10164000AA862C87CE0107960E94460786E0F801FD
:10165000ADE0B2E001900D928A95E1F70E94DC09BD
:101660000E94CE090AC05E1711F1C8010E94B1079D
:1016700081112CC0C8010E944607FF24F394D1C0F9
:10168000282F207F81F77A2DB98AA88A6E2D898923
:101690000E94B9078DE092E00E94460786E0D601DD
:1016A0001D928A95E9F70E94CE09F12CBAC0491320
:1016B000DCCFE110DACFF8018583C8010E9446072C
:1016C00086E0D6011D928A95E9F7ABC0EE2091F233
:1016D00020911202822F82958F7090E002970CF475
:1016E000B5CF80910D0290910E029A8389831B825F
:1016F000BD82AC822E83CE010196A6CF62177307FE
:1017000008F044C0FE2CEE2009F4B4CF5E1330C0C4
:1017100049132EC02091120220FD21C0822F8295F4
:101720008F70482F50E041155105C9F0F80125830D
:101730004F30510541F08F5F982F9295907F822F07
:101740008F70892B8583C8010E94460786E0F801C7
:10175000ADE0B2E001900D928A95E1F73CC086E0E1
:10176000F801ADE0B2E001900D928A95E1F759C021
:10177000C8010E94B107811169CF80911202816076
:1017800080931202C8010E9446074BC07A2DB98A85
:10179000A88A6E2D89890E94B90786E0D6011D921C
:1017A0008A95E9F718C0EE2009F464CFC8010E94B9
:1017B000B107F82E882309F45DCF86E0F801ADE08B
:1017C000B2E001900D928A95E1F78DE092E00E94DF
:1017D000B7030E94DC090E94CE0923C04D875E87B3
:1017E0008D859E850E947F09292F22952F7022309A
:1017F00028F49F7039F0811105C00BC0243028F403
:101800009F7049F4805E883020F0C8010E9446072E
:101810009F2CF92C06C0D80115969C91907F91F7CA
:10182000F8CF8F2D61960FB6F894DEBF0FBECDBFF7
:10183000DF91CF911F910F91FF90EF90DF90CF90AC
:10184000BF90AF909F9008951F93CF93DF93CDB734
:10185000DEB72C970FB6F894DEBF0FBECDBF4F8317
:10186000588769877A878B879C87CE0107960E9465
:10187000540A8823D1F09F8188852A853B85232BB4
:1018800031F08F3F31F481E09F3F19F403C081E0D4
:1018900001C080E080FD47C04F81588569857A8509
:1018A0008B859C850E94C8073EC086E0FE01379666
:1018B000DE01119601900D928A95E1F7FF81E8858E
:1018C0006A857B856115710531F0EF3F31F481E068
:1018D000FF3F19F403C081E001C080E080FD23C018
:1018E0002091DC0130E0C901019687709927409171
:1018F000DB0150E084179507F1F1F983EA837D83DA
:101900006C8396E0929FD001939FB00D1124A35257
:10191000BE4FFE01319601900D929A95E1F78093AA
:10192000DC010E94AD0916E08091DB019091DC01A1
:10193000891771F1189FC001112483529E4F0E9494
:10194000540A882329F1E091DB011E9FF001112444
:10195000E352FE4F40815181628173818481958180
:101960000E94C8078091DB0190E00196877099275B
:101970008093DB01D9CF0E9492071092DC01109274
:10198000DB01EDE0F2E086E0DF011D928A95E9F7E8
:101990002C960FB6F894DEBF0FBECDBFDF91CF916E
:1019A0001F910895809133028595859585950895B9
:1019B000809133028770089590913302977081E08F
:1019C00009F480E00895809156020895909156029E
:1019D000892B809356020895809590915602892311
:1019E00080935602089510925602089590915502E0
:1019F000892B8093550208958095909155028923F3
:101A000080935502089510925502089580913402F2
:101A1000089508950C94090D0C940A0D9091B70245
:101A200092FD08C090913402981721F080933402FF
:101A30000C940C0D089580913402882329F01092A3
:101A4000340280E00C940C0D0895CF93DF93E09165
:101A50000201F0910301809156028083E09102011E
:101A6000F0910301908180915502892B80838091B0
:101A70003402882381F0E0910201F091030190810A
:101A8000892B808380910201909103010E94B71FEE
:101A900081110E941B0DC0910201D091030140E20F
:101AA00050E063E172E0CE010E940C29892B69F0BD
:101AB00080E2FE01A3E1B2E001900D928A95E1F788
:101AC000CE01DF91CF910C94631FDF91CF910895E8
:101AD0000C94090D9091B70292FD10C098E0899F77
:101AE00090011124262B209333020E944A088091F2
:101AF00033028595859585950C94680D0C944A085C
:101B00001092330280E00C94680D2091330280958E
:101B1000822380933302982F977099F430E0482FF6
:101B2000082E000C550B2417350759F09091B70279
:101B300092FD07C08595859585950E946B080C944C
:101B4000800D08959091B70292FB222720F9281763
:101B500069F080FB92F99093B7028091B602909160
:101B6000B7020E94F00D82E00C94850D08958091DB
:101B7000B70282FB882780F991E089270C94A20D97
:101B800081E00C94A20D80E00C94A20D6FEF7FEF2A
:101B900080E090E00C944B2980E090E00E9427299F
:101BA00021E0893E9E4F09F020E0822F089582E0D7
:101BB00090E00C94192983E090E00C941929CF93BC
:101BC00084E090E00E941929C82F82E290E00E94F0
:101BD00019292C2F30E0A901582BCA01CF91089563
:101BE000CF93C92F682F84E090E00E942D296C2F9D
:101BF00082E290E0CF910C942D29AB01BC018FE0E3
:101C000090E00C943F29AB01BC0183E190E00C947F
:101C10003F2960E070E0CB010C94030E60E070E0BF
:101C2000CB010E94FD0D0C94090E69EE7EEF80E061
:101C300090E00E944B2960E082E090E00E942D2914
:101C400060E083E090E00E942D291092D70110926D
:101C5000D8011092D9011092DA0160E084E090E09E
:101C60000E942D2960E082E290E00E942D2960E030
:101C700085E090E00E942D2960E086E090E00E94DF
:101C80002D296FEF87E090E00E942D2940E050E081
:101C9000BA0188E090E00E943F2960E08DE090E08A
:101CA0000E942D2940E050E0BA0188E190E00E94B6
:101CB0003F2960E087E190E00E942D2940E050E05C
:101CC000BA018CE190E00E943F2960E070E080E280
:101CD00090E00E944B2940E050E0BA0188E190E09A
:101CE0000E943F290C940E0E0C94150E682F8EE066
:101CF00090E00C942D290E941E2160936102709344
:101D00006202809363029093640260935D02709319
:101D10005E0280935F029093600208950E941E21EC
:101D200060936102709362028093630290936402F5
:101D30006093590270935A0280935B0290935C0205
:101D4000089585B7806885BF85B7806885BF089589
:101D500081E008950C94A80E08950C94AC0E0C9498
:101D6000AC0E0C94AF0E0C94AC0E0C94B30E0C9401
:101D7000AC0E0E94A10E8BE691E10E944D1F0E94C5
:101D8000B70E0C94B50E0E94AD0E0C94AC0E0E94D2
:101D900085110C9451030E9409210E9452120E9445
:101DA000C70E0E94C31A0E94EF1D0C94B10E8F92B1
:101DB0009F92AF92BF92CF92DF92EF92FF920F93DA
:101DC0001F93CF93DF93CDB7DEB72A970FB6F89462
:101DD000DEBF0FBECDBF0E946112982E81110E94FE
:101DE0007B0E87E5A82E82E0B82E00E010E0802E62
:101DF000802F0E94A911D82EF501C1905F01C8263D
:101E0000B1F40F5F1F4F0230110589F78FEF8983FF
:101E10008A831B820E9412218160782F9D838C838C
:101E200049815A816B818D810E946D032FC0809101
:101E3000650281FD0E94AF11E12CFF24F3948C2DEB
:101E40008F21F1F00E94AA0E882399F0EE828F82F2
:101E5000DF2081E009F480E088870E941221816000
:101E6000782F9A8789874E815F8168858A850E944D
:101E70006D03F801E95AFD4F8081F826F08206C013
:101E8000E394FF0CF4E0EF12DACFBBCF81E09110C6
:101E900001C080E02A960FB6F894DEBF0FBECDBF1A
:101EA000DF91CF911F910F91FF90EF90DF90CF9036
:101EB000BF90AF909F908F9008950E94D70E0E9480
:101EC000F61A0E94081E81110E948E0E0E94511463
:101ED0000C946203CF93DF930E949410EC01811560
:101EE00021E5920708F045C0811530E5930708F019
:101EF00094C0883E910528F5803E910508F0F8C011
:101F0000883A910570F4853A910508F07CC08130DB
:101F1000910509F475C008F4E8C0049708F0E8C01A
:101F2000E4C08F3B910508F0E0C0C85AD0E0CC0F68
:101F3000DD1FC35ADE4F0990D881C02DCE019464B5
:101F4000D8C0811540E2940758F4811551E09507F7
:101F500008F0CEC08D3E910508F4C7C09065C9C099
:101F6000C11580E4D80708F4C0C0DF70CE01906AC4
:101F7000C0C0811525E59207A8F4811534E59307C3
:101F800008F095C0811543E5940708F07BC08115E2
:101F900052E5950708F061C0D82FCC27CE01816F9C
:101FA000906AA7C0C11589E5D807A0F4C11528E536
:101FB000D20708F082C0C11536E5D30708F095C0F6
:101FC0008C2F0E9428118F7190E0D82FCC27CE0142
:101FD00090628FC0C1154AE5D40708F474C0CE01E1
:101FE00090568115904208F080C08D2F8F710E940D
:101FF0002811DD27D0628F71AE01582BCA0179C03C
:1020000081E090E076C0C55AD0E0C557DE4F8881A8
:10201000C82FD0E0CE0190646CC074E0969587958F
:102020007A95E1F7282F23703C2F337081E090E000
:1020300002C0880F991F3A95E2F79C68AC01522BB9
:102040009A019C2F9F709695969550E2959FE0017E
:102050001124C9018C2B9D2B4CC08370992721E042
:1020600030E002C0220F331F8A95E2F79C2F96952D
:10207000969580E2989FE0011124C22BD32BCE01CC
:102080009C6837C08370992721E030E002C0220F9E
:10209000331F8A95E2F79C2F9695969540E2949F80
:1020A000E0011124C22BD32BCE019A6822C0D82F75
:1020B000CC27CE01846F906A1CC0DC2FCC27CE01C8
:1020C000806F906A16C08C2F8F700E94281194E048
:1020D000D695C7959A95E1F7CF70D0E0DC2FCC2745
:1020E000D0699E01282BC90104C080E090E001C0A6
:1020F000CE01DF91CF910895E72FF0E0E80FF11DB9
:10210000E80FF11DEE0FFF1FEE0FFF1FE60FF11D91
:10211000EE0FFF1FE852FF4F8591949108950E94A2
:102120007C100E946A0F08958238910569F1B0F41D
:102130008133910509F46DC048F48932910509F4A1
:1021400063C08A32910509F469C008958533910509
:1021500009F455C089339105B9F00895833E91057E
:1021600069F138F4803E9105B1F0823E910509F1A4
:102170000895863E9105A9F1873E9105B9F1843E07
:10218000910509F064C023C02091B60220FD4FC024
:1021900021FD4DC008958091B60280FD44C080911C
:1021A000B70280FF44C08091B60284FD42C083EE36
:1021B0004DC08091B60282FF38C0F5CF8091B60243
:1021C00082FD33C08091B70280FD31C0ECCF809199
:1021D000B70281FF32C08091B60284FD2AC087EE2B
:1021E00035C08091B60283FF26C0F5CF8091B6023C
:1021F00083FD21C08091B70281FD1FC0ECCF80918B
:10220000B60285FD1CC01DC08091B60285FD19C0B7
:1022100016C08091B60286FD16C017C08091B60226
:1022200086FD13C010C089E311C082EE0FC080EE9E
:102230000DC080E00BC086EE09C084EE07C089E2C5
:1022400005C085E303C08AE201C081E390E0089500
:102250009091B60292FF0DC0282F2871283019F4F2
:10226000877F846006C0282F2471243011F48B7F6F
:10227000886093FF0DC0282F2871283119F4877EBC
:10228000846106C0282F2471243111F48B7E88616B
:102290002091B70220FF0DC0382F3871383019F463
:1022A000877F816006C0382F3171313011F48E7F05
:1022B000886021FF0DC0282F2871283119F4877EEE
:1022C000816106C0282F2171213111F48E7E886131
:1022D00094FD877E089580E008950C94C60D0E94B9
:1022E00061128FE39CE90197F1F700C000000E94A2
:1022F000611280E00E94A91180FF04C00E946D114C
:102300000C945F2108950C946F110E94CC0D8111E3
:1023100002C00E94740E0E94D70D809365020E9435
:10232000DF0D9093B7028093B6020E9483110E9442
:10233000DB0D682F70E080E090E00E94EA0760917A
:10234000D3017091D4018091D5019091D6010C9464
:102350002208E82FF0E0E654FD4F808108950895AB
:1023600080EA8A95F1F7089500C008950C94B011A1
:1023700008950C94B8110C94B9110C94B8110C94E4
:10238000BD11F894E82FE295EF70F0E031A1282F0D
:102390002F7081E090E001C0880F2A95EAF7982F0E
:1023A0009095932391A392A1892B82A37894089569
:1023B000CF93DF9387E60E94C11186E60E94C11188
:1023C000CEE8D1E089918F3F11F00E94C11181E0E8
:1023D000C239D807B9F7DF91CF910895CF92DF9234
:1023E000EF92FF920F931F93CF93DF938C01C62F31
:1023F000D0E0CE018E569E4F7C01FC0190819F3F24
:1024000009F447C0D62EF894E92FE295EF70F0E07A
:1024100081A19F7021E030E001C0220F9A95EAF778
:10242000822B81A382A12095282322A378940E9445
:10243000B411EEE8F1E042E951E031E0C12C219124
:102440002F3F89F0A22FA295AF70B0E090968C91AB
:1024500090E02F7002C0959587952A95E2F780FD50
:1024600002C0832F01C080E0C82A330F4E175F07D8
:1024700031F7F70180818F3F11F00E94C11161E0B7
:10248000C11001C060E08D2D0E94B611C00FD11F98
:10249000C882DF91CF911F910F91FF90EF90DF9055
:1024A000CF9008950E94D8111092BB021092BA02E8
:1024B0001092B9021092B80282E00E9499120C9414
:1024C000D5021F93CF93DF9300D0CDB7DEB71A822A
:1024D000198260E0CE0101960E94EE1161E0CE010A
:1024E00001960E94EE1142E050E0BE016F5F7F4F07
:1024F00088EB92E00E940C2911E0009709F410E0AB
:10250000892B31F089819A819093B9028093B80226
:10251000212F42E06AEB72E088EB92E00E949A126F
:102520000E94D702812F0F900F90DF91CF911F91C2
:1025300008950895FF920F931F93CF93DF938C011B
:10254000F62ED72FC42F222349F081E08093680212
:102550000E94122190936702809366028091680224
:102560008823C1F080916602909167020E942A211F
:10257000059780F0EF2DFD2FD8014C2F50E0CD01B5
:10258000801B910B841795071CF48D918193F7CFD5
:1025900010926802DF91CF911F910F91FF900895E3
:1025A0000E942A230E94CB0E0C9436230E943A23C9
:1025B0000E945D0F0C9454230E94B0200E941123AE
:1025C0000E94B90E0E94D0120E94D6120E94C30E21
:1025D000FBCF80916F0280FF06C06091090170E01F
:1025E000660F771F26C081FF04C06091090184E057
:1025F00005C082FF07C06091090188E0689FB001B3
:10260000112417C090916E029923D1F060910801B6
:10261000961788F72091090188E0289F90011124DE
:10262000929FA001939F500D112470E0CA010E9457
:1026300086286038710540F46115710519F406C0EB
:1026400068E070E0862F08958FE7089581E008958F
:1026500080916F0280FF08C06091050170E0759560
:1026600067957595679521C081FF06C0609105014A
:1026700070E07595679519C082FF04C060910501EF
:1026800070E010C090916D02992399F0609104015F
:102690009617A0F780910501899FC001112470E071
:1026A0000E9486286038710540F46115710519F49F
:1026B00006C061E070E0862F08958FE7089581E0FD
:1026C00008958D3E21F40E94E912819504C08E3E4A
:1026D00029F40E94E9128093730208958F3E21F439
:1026E0000E94E912819504C0803F29F40E94E912FA
:1026F000809372020895893F19F40E94281305C03F
:102700008A3F31F40E9428138195809374020895C2
:102710008B3F21F40E942813819504C08C3F29F43B
:102720000E9428138093750208959FE0980F9830B7
:1027300078F421E030E0A90102C0440F551F9A95BA
:10274000E2F7CA0190917102892B8093710208957A
:102750008D3F21F480916F0281600BC08E3F21F488
:1027600080916F02826005C08F3F29F480916F02D3
:10277000846080936F0208958D3E39F490917302C6
:1027800097FF35C01092730259C08E3E29F4909184
:1027900073021916BCF32BC0909172028F3E29F47C
:1027A00097FF25C01092720249C0803F19F4191694
:1027B000CCF31DC090917402893F29F41916BCF422
:1027C000109274023BC08A3F19F497FF10C0F8CFF3
:1027D0008B3F39F49091750297FF09C010927502F2
:1027E0002DC08C3F21F4909175021916BCF39FE027
:1027F000980F983080F421E030E0A90102C0440F26
:10280000551F9A95E2F7CA0180959091710289232C
:102810008093710213C08D3F21F480916F028E7FEF
:102820000BC08E3F21F480916F028D7F05C08F3FDA
:1028300029F480916F028B7F80936F0280917202E6
:10284000811106C080917302811102C010926E0244
:1028500080917402811106C080917502811102C0BD
:1028600010926D0208950E9412212091720221118E
:1028700004C020917302222321F090936C02809374
:102880006B0220917402211104C020917502222351
:1028900021F090936A028093690280E792E00C94A1
:1028A0007D1FEF92FF920F931F93CF93DF9300D082
:1028B00000D000D0CDB7DEB786E0E0E7F2E0DE0181
:1028C000119601900D928A95E1F7E0907202F090D6
:1028D00073020091740210917502109272021092AC
:1028E00073021092740210927502E11003C0FF206F
:1028F00009F45DC080916B0290916C020E942A21C4
:10290000AC0190916E02992339F020910A0130E0D8
:102910002417350758F04BC020910B018AE0289FFF
:10292000900111242417350718F041C09F3F19F07A
:102930009F5F90936E02EE2061F00E94E9121E14D8
:1029400014F09FEF01C091E0989F902D1124909377
:102950007202FF2061F00E94E9121F1414F09FEF31
:1029600001C091E0989F902D1124909373023091B3
:1029700072023323E1F0209173022223C1F045EB70
:102980003403C0011124992319F09093720203C0FB
:1029900081E08093720235EB2303C0011124992357
:1029A00019F09093730203C081E0809373020111C8
:1029B00003C0112309F45DC08091690290916A02FD
:1029C0000E942A21AC0190916D02992339F0209147
:1029D000060130E02417350758F04BC0209107015D
:1029E0008AE0289F900111242417350718F041C070
:1029F0009F3F19F09F5F90936D02002361F00E944A
:102A00002813101614F09FEF01C091E0989F902DAD
:102A1000112490937402112361F00E94281311165F
:102A200014F09FEF01C091E0989F902D1124909396
:102A30007502309174023323E1F020917502222354
:102A4000C1F045EB3403C0011124992319F0909390
:102A5000740203C081E08093740235EB2303C0014C
:102A60001124992319F09093750203C081E080939B
:102A700075028091720281110BC0809173028111E5
:102A800007C080917402811103C080917502811189
:102A90000E943314EB82FC820D831E8386E0FE01CC
:102AA0003196A0E7B2E001900D928A95E1F7269663
:102AB0000FB6F894DEBF0FBECDBFDF91CF911F914F
:102AC0000F91FF90EF900895E0E7F2E086E0DF01DC
:102AD0001D928A95E9F710926E0210926D02109283
:102AE0006F020895EF92FF920F931F93CF93DF939E
:102AF0008B01682F11110AC0442329F0E82FF0E060
:102B0000E15FFD4F6491762F862F75C0212F30E055
:102B1000E82FF0E0442321F0E15FFD4FE491F0E085
:102B200046E0049FC0011124CFEFD0E0BE010E9417
:102B300072284BEA4603C001479F900D1124800F75
:102B4000911D800F911D982F990F890FAE01421B87
:102B5000530B4E9FD0014F9FB00D5E9FB00D1124BF
:102B60009B2F189FA0011124452F55278E01041B70
:102B7000150B0E9FA0010F9F500D1E9F500D11248D
:102B80007E01E81AF108E29E8001E39E100DF29E9C
:102B9000100D1124212F3327C21BD30BCE9F900180
:102BA000CF9F300DDE9F300D112462307105A9F0EA
:102BB00048F46115710569F061307105C9F48B2F16
:102BC000752F0DC06430710581F058F066307105C5
:102BD00079F47E2F8B2F932F0DC0832F7B2F9E2F69
:102BE00009C08E2F7B2F952F05C08E2F732F02C00B
:102BF0007E2F852F692FDF91CF911F910F91FF902D
:102C0000EF90089541E00E947215089508950E9482
:102C100002160895CF93DF93762FE901682F842F52
:102C20000E940716798368838A83DF91CF91089584
:102C30008091BC02282F269530E02115310519F42A
:102C40008170826005C02532310524F0817088646E
:102C50008093BC02089588E090E00C942129CF92E3
:102C6000DF92EF92FF926B017C010E941816B70170
:102C7000A60188E090E0FF90EF90DF90CF900C9459
:102C80003F29ECEBF2E083E0808311828FEF8283B7
:102C90008383148260817181828193810C942F16C9
:102CA0008091BC0280FF02C08695089580E008955F
:102CB0009091C002933018F49F5F9093C0028823D4
:102CC00051F06091BC027091BD028091BE02909162
:102CD000BF020C942F16089581E00C945816909121
:102CE000C002992319F091509093C002882351F0AB
:102CF0006091BC027091BD028091BE029091BF02B2
:102D00000C942F16089581E00C946F1670E00C94CB
:102D1000731C609110018091BC0280FF0AC08091F9
:102D20000F0123E0829FC00111248F539D4F0C940B
:102D300086168091110190911201891780F7E82F72
:102D4000F0E09F01220F331FE20FF31FEF53FD4FFF
:102D50001182108212828F5FF0CF9091BC0290FF9F
:102D600016C09091110120911201921770F4E92F71
:102D7000F0E0DF01AA0FBB1FEA0FFB1FEF53FD4F6F
:102D80008183608342839F5FF0CF0C9489160895FE
:102D9000CF93DF9300D01F92CDB7DEB79091BC02E6
:102DA00090FF0AC09E012F5F3F4F0E940A164B8181
:102DB00069818A810E94AD160F900F900F90DF916C
:102DC000CF910895CF93DF93EC01EC81F0E0E65FC3
:102DD000FE4F4491ECEBF2E0628181810E94C816C3
:102DE0008C818F5F8C83DF91CF910895CF93DF9398
:102DF000EC01ECEBF2E0438162818C810E94C81609
:102E00008C818F5F8C83DF91CF9108950F931F93F7
:102E1000CF93DF9300D01F92CDB7DEB78C018091A6
:102E2000760281110AC09E012F5F3F4F4FEF6FEF77
:102E30000E940A168A8180937602F801848181308B
:102E400051F028F0823061F4409176020AC08091FE
:102E5000760240E007C06091760240E080E003C067
:102E600040E080E060E00E94AD16F801848190E0CF
:102E7000019663E070E00E94862884830F900F9093
:102E80000F90DF91CF911F910F910895AF92BF9254
:102E9000CF92DF92EF92FF920F931F93CF93DF9326
:102EA00000D01F92CDB7DEB7182FF62E042FE22EDA
:102EB0009091BC0290FF6DC0E92FE695AE2FB0E077
:102EC000AC56BE4F8C91809380029E7F923061F40D
:102ED0009E012F5F3F4F812F0E940A164B8169810F
:102EE0008A810E94AD1643C0823019F40091BF025E
:102EF0003EC0863019F41091BD0239C08930D9F333
:102F00008931A9F5E9518E2F8170D82EE695F0E030
:102F1000E65FFD4FA590B490C12CBB2460911301D6
:102F2000C61618F52C2D30E0A29EC001A39E900D70
:102F3000B29E900D112470E00E947228812FD11052
:102F400002C0860F01C0861B90911101290F311D0F
:102F5000A901440F551F240F351F2F533D4F402FFC
:102F60006F2D0E940A16C394D9CF0E948916109320
:102F7000BD02F092BE020093BF02EE2051F06091BC
:102F8000BC027091BD028091BE029091BF020E946E
:102F90002F160F900F900F90DF91CF911F910F91EF
:102FA000FF90EF90DF90CF90BF90AF900895ECEB43
:102FB000F2E09181282F4381628188E0890F0C948F
:102FC000461781E00C94D717ECEBF2E09181282FA3
:102FD0004381628188EF890F0C94461781E00C943D
:102FE000E417ECEBF2E0628121E1620F08F46FEF8D
:102FF000282F438181810C94461781E00C94F117AE
:10300000ECEBF2E0628121E1621B08F460E0282F22
:10301000438181810C94461781E00C940018ECEBFD
:10302000F2E0438121E1420F08F44FEF282F628143
:1030300081810C94461781E00C940F18ECEBF2E0C0
:10304000438121E1421B08F440E0282F6281818105
:103050000C94461781E00C941E1820E00C9446173F
:10306000FF920F931F93CF93DF93EC01F12C0FEF9F
:1030700010E060911301F616F0F4809111012F2DEC
:1030800030E0280F311DC901880F991F280F391F03
:103090002F533D4F70E0C8010E948628962F8C81E7
:1030A0004091BF026091BE02F99E800D11240E94E2
:1030B0000A16F394DECF0E9489169A818C8190FFC4
:1030C00002C08F5F01C081508C83DF91CF911F912F
:1030D0000F91FF900895AF92BF92CF92DF92EF923F
:1030E000FF920F931F93CF93DF93FC01828180FFA8
:1030F00002C00FEF01C001E010E043E0A42E809178
:103100001301181708F043C080911101C12ED12C72
:10311000E601C80FD11DCE01880F991FC80FD91F16
:10312000CF53DD4F198218821A8234E0E32EF12C3E
:10313000B12C809178028B0D84302CF06A2D0E9486
:103140006428892F05C087FF03C090911301890F60
:10315000082E000C990BC816D90691F48091BF0275
:103160008E9DA0018F9D500D112455954795559525
:1031700047959E016091BE028091BD020E940A1691
:10318000B00EF1E0EF1AF108A1F61F5FB8CF0E9470
:10319000891680917802013031F4811102C080914A
:1031A0001301815007C090E001966091130170E017
:1031B0000E94862880937802DF91CF911F910F9112
:1031C000FF90EF90DF90CF90BF90AF900895CF9396
:1031D0008091110190911201891770F4E82FF0E0AD
:1031E0009F01220F331FE20FF31FEF53FD4F118298
:1031F000108212828F5FF0CFC0E060911301C6177A
:10320000C0F5EC2FF0E070E0CF010E9486282091FD
:103210001101820F20917702022E000C330B90E0F7
:10322000E217F307CCF020910E01022E000C330BB5
:103230002E173F078CF09C01220F331F820F931F24
:103240009C012F533D4F4091BF026091BE0280917F
:10325000BD020E940A160BC0FC01EE0FFF1F8E0F6D
:103260009F1FFC01EF53FD4F118210821282CF5F2E
:10327000C4CF0E94891620910D0180917702820FA0
:103280008093770290910E01920F90930E01191680
:103290005CF4082E000C990B4091130150E0415052
:1032A0005109841795071CF0219520930D01CF91AA
:1032B00008958F929F92AF92BF92CF92DF92EF923A
:1032C000FF920F931F93CF93DF938C01FC014481F6
:1032D000C42FD0E09E01DE010E94CA289B01AC01F0
:1032E0000E94E0286B017C01E0E2F0E0EC1BFD0BAA
:1032F000A5E5B0E09B01AC010E94E0284B015C0118
:103300009F01DF010E94C2289B01AC010E94EB28B3
:103310009B01AC012C0D3D1D4E1D5F1DC501B4016F
:103320000E949A28C22FD22F2A3228F4F3E02F9F2E
:10333000900111240DC025E530E02C1B3109C90195
:10334000880F991F280F391F37FF02C02F5F3F4F8B
:1033500035952795C22FC095F12C85E5E82EED1AFD
:1033600080911301F816C8F4F1FC02C08E2D01C043
:103370008D2F909111012F2D30E0290F311DA901C2
:10338000440F551F240F351F2F533D4F4C2F609175
:10339000BE020E940A16F394E3CF0E948916F80138
:1033A0008481811102C091E003C0803219F49FEF43
:1033B00090930C0190910C01890FF8018483DF91A7
:1033C000CF911F910F91FF90EF90DF90CF90BF9022
:1033D000AF909F908F9008950F931F93CF93DF939B
:1033E000EC0100E010E080911301282F30E002177B
:1033F000130724F5909111019801290F311DA9019E
:10340000440F551F240F351F2F533D4F869590E0D5
:103410004C81081719071CF4442331F002C04111F4
:1034200003C04091BF0201C040E06091BE028091A4
:10343000BD020E940A160F5F1F4FD5CF0E9489164A
:103440008C8190E00196817099278C83DF91CF91D8
:103450001F910F910895ECEBF2E080818E7F8083C5
:1034600060817181828193810E942F161092810266
:103470002FEF80E792E0215080409040E1F700C0BC
:1034800000000C9489166091BC02669570E04BE0D8
:1034900050E084E191E00E94FF28892B19F481E03B
:1034A000809381020E94122190937A028093790284
:1034B00008959091BC0290FF35C09170811102C0B7
:1034C000926006C0853210F0986402C0880F982B75
:1034D0009093BC02662351F06091BC027091BD02D2
:1034E0008091BE029091BF020E942F166091BC0293
:1034F000669570E04BE050E084E191E00E94FF2887
:10350000892B19F01092810202C00E94431A81E0B7
:1035100080937C024091BF026091BE028091BD0207
:103520000C942D180895682F9091BC02969581E017
:10353000890F853208F081E00C94591A81E00C94CF
:10354000931A682F9091BC0296958FEF890F09F41A
:1035500084E20C94591A81E00C94A11A61E00C9455
:10356000591AECEBF2E080818160808386950C949F
:10357000AE1A8091BC0280FD0C942B1A0C94B11AE7
:1035800060E00C94591A80917F0281112EC00E9434
:10359000CC0D811104C00E94740E0E9441160E943D
:1035A0002B166093BC027093BD028093BE02909371
:1035B000BF026E7F61F40E9441160E942B16609339
:1035C000BC027093BD028093BE029093BF020E9422
:1035D0001816109281028091BC0280FF03C086956C
:1035E0000E94C01A81E080937F0208950F931F9379
:1035F000CF93DF9380918102882309F485C0809165
:103600008002E091BC02E695E81BE0937B028230E9
:1036100049F4F0E0EA5FFE4FE491CE2FD0E002EEF5
:1036200016E149C0863049F4F0E0ED5FFE4FE491C9
:10363000CE2FD0E006EF16E13EC0893051F4E6957A
:10364000F0E0E050FF4FE491CE2FD0E000E318E12E
:1036500032C08F3051F4E695F0E0E350FF4FE49133
:10366000CE2FD0E00BE618E126C0853149F4F0E01A
:10367000E650FF4FE491CE2FD0E007EE18E11BC0DB
:10368000883181F0833239F4E8EFF0E0C591D491CC
:1036900006E017E110C0843251F4C4EFD1E00CEE23
:1036A00019E109C0C8E2D0E009E519E104C0C0EDA4
:1036B000D7E006E016E180917C02882361F0109249
:1036C0007C020E94122190937A02809379021092D8
:1036D0007E0210927D020E941221E0917902F09107
:1036E0007A028E1B9F0B8F3F9F4770F4EC0FFD1FDC
:1036F000F0937A02E093790289E792E0F801DF9192
:10370000CF911F910F910994DF91CF911F910F914C
:103710000895882311F0FA0101C0FB010994CF93A9
:10372000DF93C82FD62F0E9450168C1740F00E94AE
:1037300050168D1720F4DF91CF910C949E1A8C2F88
:10374000DF91CF910C94AE1A1F93CF93DF93FB01BF
:1037500012811111C3C0EC010E94E30C8272CD3CB6
:10376000FCE5DF0709F49AC0A8F5C73CECE5DE07E5
:1037700009F476C0A8F4C43C9CE5D90709F45FC0FD
:1037800028F4C33CDC4509F457C054C0C53C9CE553
:10379000D90709F459C0C63CDC4509F45CC04AC0ED
:1037A000CA3CFCE5DF0709F46AC050F4C83CECE50C
:1037B000DE0709F45AC0C93CDC4509F45BC03AC0D5
:1037C000CB3C9CE5D90709F45FC0CC3CDC4509F44F
:1037D00060C030C0C23DFCE5DF0709F46FC088F46B
:1037E000CF3C9CE5D90709F460C008F45CC0C03D3B
:1037F000FCE5DF0709F45CC0C13DDC4509F45BC0B2
:1038000019C0C53D9CE5D90709F460C050F4C33D1B
:10381000FCE5DF0709F455C0C43DDC4509F454C09C
:1038200009C0C63D9CE5D90709F455C0CE35DD4534
:1038300009F454C011E052C00E94B91A4FC04BEABB
:103840005AE16EE97AE104C04EE95AE16BEA7AE1A5
:103850000E94891B43C04EEE57E161EE77E1F8CF3D
:1038600041EE57E16EEE77E1F3CF4CE058E16DEFBA
:1038700077E1EECF4DEF57E16CE078E1E9CF4AE236
:1038800058E16BE178E1E4CF4BE158E16AE278E19D
:10389000DFCF43E856E16CE676E1DACF4CE656E15D
:1038A00063E876E1D5CF81E017C065E082E010C023
:1038B00068E086E00DC06EE089E00AC064E18FE058
:1038C00007C067E185E104C088E106C062E289E1E2
:1038D0000E948F1B03C083E20E94AE1A812FDF91EA
:1038E000CF911F910895269A25B12F7B35B1306471
:1038F0004FB7F894FC01CB01880F991F680F791F0F
:103900006E0F7F1FE617F70789F0819198E035B9B0
:10391000000000C087FF25B9880F000000C000C06C
:1039200000C025B900C09A9591F7ECCF4FBF8FE545
:1039300094E00197F1F700C000000895CF93DF9362
:10394000EC01FB018281882309F43CC1C430FDE510
:10395000DF0760F4CB3F9CE5D90788F49E01225035
:103960003C452431310508F02EC109C0C236EDE5D1
:10397000DE0729F0C63AFDE5DF0709F024C10E9401
:10398000DF0D9093B7028093B602C1318CE5D80762
:1039900009F4C6C008F042C0C930ECE5DE0709F4FE
:1039A0009BC000F5C5308CE5D80709F485C078F4D4
:1039B000C330ECE5DE0709F478C008F07AC0C23005
:1039C000DC4509F0F5C08091B6028160EFC0C730D8
:1039D0009CE5D90709F478C008F07AC08091B60256
:1039E0008061E4C0CD30FCE5DF0709F487C058F4FE
:1039F000CB309CE5D90709F479C008F07BC08091F1
:103A0000B60288606FC0CF30FCE5DF0709F480C0E4
:103A100008F082C08091B602877FC8C0CE3F9CE587
:103A2000D90709F471C000F5C531FCE5DF0709F4D9
:103A300085C068F4C3319CE5D90709F475C008F066
:103A400095C00E9492078091B6028F77AFC0CC3F9D
:103A5000FCE5DF07A9F108F054C0CB3FDC4509F0D5
:103A6000A7C08091B70240C0C230EDE5DE0709F47F
:103A700089C058F4C1158DE5D80709F45AC008F07B
:103A800069C08091B70282602FC0C236EDE5DE07C3
:103A900009F47CC0C63AFDE5DF0709F481C0C330F4
:103AA000DD4509F085C080E06EC08091B60282607D
:103AB0007DC08091B60216C08091B602886076C043
:103AC0008091B70282604FC08091B60280626EC062
:103AD0008091B60280646AC00E9492078091B6020B
:103AE000806864C0846062C081603DC08091B6021D
:103AF0008E7F5CC08091B6028D7F58C08091B602E7
:103B000016C08091B70218C08091B7028D7F2BC07C
:103B10008091B6028F7E4AC08091B6028F7D46C0EA
:103B20008091B6028F7B42C08091B602877F8B7FE7
:103B30003DC08091B7028D7F8E7F15C08091B60207
:103B400082FB222720F991E0922790FB82F990FBDB
:103B500083F92CC08091B702982F909591708E7F39
:103B6000892B90FB81F98093B70222C00E949207B3
:103B70008091B60287FB222720F991E0922790FBE3
:103B800087F914C081E00E94760E12C08091B602BF
:103B900084FB222720F991E0922790FB84F906C04C
:103BA0008091B602982F909590FB80F98093B60291
:103BB0008091B6029091B7020E94F00D0E94920788
:103BC00080E001C081E0DF91CF9108958FE891E01E
:103BD0000197F1F700C0000008950C947802569800
:103BE0005E9A57985F9A0E94E61D89B186FB8827E6
:103BF00080F929B130E0220F232F221F330B232B12
:103C000011F490E001C092E0892B80938402089522
:103C1000E0918402EE0FEE0FE093840229B126FBBF
:103C2000882780F990E029B130E0220F232F221F4E
:103C3000330B2115310511F022E030E0822B932B5C
:103C40008E2B809384028F70E82FF0E0E754FE4FB4
:103C5000908180918302890F8093830284305CF08D
:103C6000809182028F5F8093820260E080E00E94F8
:103C7000ED1D21E001C020E0809183028D3F54F4CE
:103C80008091820281508093820261E080E00E94F4
:103C9000ED1D21E080918302082E000C990B64E059
:103CA00070E00E94862880938302822F0895CF932C
:103CB000DF9386319C4541F5EB010E94E30C982F80
:103CC0008A812091020130910301882379F09A7A48
:103CD00081E009F480E080938502911102C069E2DD
:103CE00001C065E3C9010E944D200AC08091850290
:103CF000811102C069E201C065E3C9010E94582038
:103D00000E94250D80E001C081E0DF91CF910895F0
:103D10000F931F93CF93DF93C42FD22FFC01828187
:103D20008823C9F0409388020E9412219093870251
:103D30008093860280E28C0F883008F057C0C770ED
:103D400081E001C0880FCA95EAF7DF91CF911F91FA
:103D50000F910C94EF0480918802481330C0809139
:103D60008602909187020E942A21883C910538F5AD
:103D700010E21D0FCD17B9F080E28C0F883040F4AF
:103D8000C77081E001C0880FCA95EAF70E94F60467
:103D9000183028F581E09D2F977001C0880F9A9503
:103DA000EAF70E94EF04802F0E94E6041830F0F436
:103DB000D77081E001C0880FDA95EAF70AC080E287
:103DC0008C0F883098F4C77081E001C0880FCA95C5
:103DD000EAF7DF91CF911F910F910C94F604802F99
:103DE000DF91CF911F910F910C94E604DF91CF9159
:103DF0001F910F9108950F939C01CB01243F4CE537
:103E0000340731F188F4293DFCE53F07D9F02A3D1C
:103E10004CE5340779F1283D3C45A9F506E221EE51
:103E200041EE68ED7CE52BC0263FFCE53F07E1F065
:103E3000A8F0273F3C4539F507E225EE46EE67EF4F
:103E40007CE51DC007E225EE45EE69ED7CE517C077
:103E500006E221EE40EE64EF7CE511C007E225EEBC
:103E600044EE65EF7CE50BC006E221EE42EE66EF24
:103E70007CE505C008E221E045EE6AED7CE50E94A4
:103E8000881E80E008C0FC018281882319F010920E
:103E9000880201C081E00F9108959093CB01809337
:103EA000CA01089590938E0280938D020895E09147
:103EB0008D02F0918E02309721F00190F081E02D7B
:103EC000099480E00895E0918D02F0918E02309780
:103ED00099F020912B01222359F02091B60227FF5F
:103EE00007C0DC012C9111962C93119726E02C939E
:103EF0000280F381E02D09940895E0918D02F09104
:103F00008E02309739F022E0DC012C930480F58199
:103F1000E02D0994089520918B0230918C0228178E
:103F2000390771F090938C0280938B02E0918D029F
:103F3000F0918E02309721F00680F781E02D0994F0
:103F400008952091890230918A022817390771F06B
:103F500090938A0280938902E0918D02F0918E0203
:103F6000309721F00084F185E02D09940895FC013B
:103F7000329680912B01882331F08091B60287FF21
:103F800002C09EE101C096E080E0915028F02191AE
:103F90002223D9F38F5FF9CF0895662351F1209141
:103FA0002B012223E9F02091B60227FF19C0462FEA
:103FB0004695469546954E31E0F4677021E030E035
:103FC00002C0220F331F6A95E2F7FC01E40FF11DD6
:103FD000828190E02823392381E0232B69F409C0F2
:103FE000FC01329608962191621729F0E817F9072B
:103FF000D1F780E0089581E008959C01FC0132969C
:104000009FEF80E04191461789F09F3F19F44111DD
:1040100001C0982F8F5F8630A9F79F3F39F0F901D3
:10402000E90FF11D97FDFA956283089508959C01AB
:104030002A5F3F4FFC014281461301C01282019664
:1040400082179307B9F70895262F2695269526956A
:104050002E3168F4FC01E20FF11D677021E030E0C1
:1040600001C0220F6A95EAF78281282B22830895E6
:10407000262F2695269526952E3170F4FC01E20F09
:10408000F11D677021E030E001C0220F6A95EAF768
:104090002095828128232283089520912B012223B9
:1040A00029F02091B60227FD0C9424200C94FD1FCA
:1040B00020912B01222329F02091B60227FD0C9498
:1040C00038200C94172020912B01FC0132962223DA
:1040D00031F08091B60287FF02C08EE101C086E018
:1040E000DF011D928A95E9F7089508950C947520D3
:1040F00083E080938F020C947620811102C081E0CE
:1041000001C082E080938F020C9476200C947D2075
:1041100081E080938F020C9476200C94882008957F
:104120000C948F200C9490200C948F200C948F2052
:104130000C948F200E9496200E9461120E9494206D
:1041400080E00E94A911811108C081E00E94A9119C
:1041500091E0811103C090E001C091E0892F0895A2
:1041600008951F920F920FB60F9211248F939F9371
:10417000AF93BF9380919002811113C08091CA02C6
:104180009091CB02A091CC02B091CD024196A11D9D
:10419000B11D8093CA029093CB02A093CC02B0933E
:1041A000CD02BF91AF919F918F910F900FBE0F9055
:1041B0001F9018958091D202843031F10E94420301
:1041C0001092900220E488E190E00FB6F894A89550
:1041D000809360000FBE2093600083B7817F84606E
:1041E00083BF83B7816083BF7894889583B78E7FC0
:1041F00083BF0FB6F894A895809160008861809382
:104200006000109260000FBE08950E9492070C9407
:10421000460382E084BD93E095BD9AEF97BD8093FD
:104220006E0008952FB7F8948091CA029091CB0246
:10423000A091CC02B091CD022FBF08952FB7F89472
:104240006091CA027091CB028091CC029091CD0214
:104250002FBF08959C014FB7F8948091CA029091A6
:10426000CB02A091CC02B091CD024FBF821B930B29
:10427000089578941F920F920FB60F9211248F9386
:104280009F93AF93BF938091CA029091CB02A0916C
:10429000CC02B091CD020196A11DB11D8093CA023E
:1042A0009093CB02A093CC02B093CD02BF91AF917B
:1042B0009F918F910F900FBE0F901F90189581E0E6
:1042C0008093E00080E28093D8001092C9008FE1D3
:1042D0009EE40197F1F700C0000087E090EBDC015D
:1042E0008093DB029093DC02A093DD02B093DE02A8
:1042F0009CE088E10FB6F894A895809360000FBE0B
:1043000090936000FFCF8091B4020895089522E059
:104310002093E9002FEF3091E800215035FD06C0D1
:1043200035ED3A95F1F700002111F5CF2091E80025
:1043300025FF0BC040E050E066E070E00E94C6231D
:104340008091E8008E778093E8000895CF93DF9303
:1043500020912B01222339F02091B60227FF03C0C0
:1043600060E222E002C068E021E02093E9002FEF44
:104370003091E800215035FD06C035ED3A95F1F752
:1043800000002111F5CF2091E80025FF1DC0EC01B0
:1043900080912B01811105C040E050E068E070E0A1
:1043A00003C070E040E050E0CE010E94C62380913F
:1043B000E8008E778093E80080E2FE01A4E9B2E095
:1043C00001900D928A95E1F7DF91CF910895809346
:1043D000910270939302609392028091D202843092
:1043E00001F582E08093E9008FEF9091E800815021
:1043F00095FD06C095ED9A95F1F700008111F5CF76
:104400008091E80085FF0DC040E050E063E070E07F
:1044100081E992E00E94C6238091E8008E77809324
:10442000E8000895BC0184E00C94E721BC0183E01E
:104430000C94E7218091D102811109C00E94572577
:104440000E94B4258091E20084608093E200089588
:104450001092D10208950C948D206091CE0281E0DB
:10446000611101C080E00C9478209091D20281E02B
:10447000943009F080E06091CE020C947D2042E0FF
:1044800061EC81E00E94D02442E261EC82E00E9473
:10449000D0249091D20281E0943009F080E06091C4
:1044A000CE020C9486208091D402833009F461C03E
:1044B00030F4813071F0823009F49AC008958A3066
:1044C00009F486C08B3009F46CC0893009F0A8C0AB
:1044D00020C08091D302813A09F0A2C08091E80007
:1044E000877F8093E8008091D7029091D802892B32
:1044F00021F460E284E992E003C060E080E090E0B3
:1045000070E00E9411248091E8008B778093E8008E
:1045100008958091D302813209F082C08091D70240
:104520009091D802029708F07BC08091E800877FC5
:104530008093E8008091E80082FD05C08091D2025E
:104540008111F8CF6DC02091F3008091F20090E0CE
:10455000922B029731F48091F100813011F0863076
:1045600021F48091F1008093B4028091E8008B7770
:1045700053C08091D302813A09F052C08091D70292
:104580009091D802892B09F04BC08091E800877F79
:104590008093E8008091E80080FFFCCF80912B01A0
:1045A00036C08091D3028132D9F58091D7029091A3
:1045B000D802892BA9F58091E800877F8093E800D5
:1045C0000E9405258091D50280932B010C949207BF
:1045D0008091D302813221F58091E800877F80931A
:1045E000E8000E9405258091D6028093B5020895C7
:1045F0008091D302813AA1F48091E800877F809373
:10460000E8008091E80080FFFCCF8091B5028093A4
:10461000F1008091E8008E778093E8000C940525E6
:10462000089584B7877F84BF0FB6F894A8958091CA
:104630006000886180936000109260000FBE90E07F
:1046400080E80FB6F89480936100909361000FBEEC
:104650000C9488200E9457250E94B425E2EEF0E0D9
:1046600080818460808378940C9449288FE191E064
:104670000C94521F8091D2028530A9F48091D2020D
:10468000853079F40E94DA208091D0028823B1F33A
:104690000E949A20882391F30E94B0230E949207DF
:1046A000EDCF0C940521089508950C945723292FDC
:1046B000332723303105C9F060F42130310581F012
:1046C0002230310509F044C08BE390E029E333E068
:1046D00043C021323105E1F02232310549F138C0C1
:1046E00082E190E024E733E037C0992781309105DB
:1046F00049F028F0029761F5EFE0F3E005C0E5E34B
:10470000F3E002C0EBE1F3E0849190E09F0124C06C
:104710006115710541F061307105D1F489E090E0D7
:1047200024E633E019C089E090E02BE433E014C0C4
:104730006115710541F06130710551F486EB90E02F
:1047400026E833E009C080E490E02CE334E004C0C4
:1047500080E090E020E030E0FA013183208308958A
:1047600080E189BD82E189BD09B400FEFDCF809161
:10477000D8008F7D8093D8008091E0008260809384
:10478000E0008091E00081FDFCCF0895CF92DF92A0
:10479000EF92FF920F931F93CF93DF93EC018B0166
:1047A0007A010E942425811133C0E114F10439F00B
:1047B000F70180819181081B190BC80FD91FC12CEB
:1047C000D12C0115110519F18091E80085FD16C065
:1047D0008091E8008E778093E800E114F10449F0BD
:1047E000F70180819181C80ED91ED182C08285E0F7
:1047F0000FC00E942425882321F30AC08991809349
:10480000F10001501109FFEFCF1ADF0ADACF80E083
:10481000DF91CF911F910F91FF90EF90DF90CF909C
:1048200008952091D9023091DA022617370748F00F
:104830006115710539F42091E8002E772093E80086
:1048400001C0B901FC0120E06115710579F1809189
:10485000D2028823F1F18530F1F18091E80083FDE7
:104860003CC08091E80082FD2EC08091E80080FF6E
:10487000EBCF2091F3008091F20090E0922B611534
:10488000710551F08830910538F421912093F100A1
:10489000615071090196F3CF21E0089709F020E0FB
:1048A0008091E8008E778093E800CECF2111CFCFA2
:1048B0000AC08091D202882361F0853061F0809136
:1048C000E80083FD0AC08091E80082FFF2CF80E01B
:1048D000089582E0089583E0089581E0089520918D
:1048E000D9023091DA022617370748F061157105B1
:1048F00039F42091E8002E772093E80001C0B90137
:10490000FC0120E06115710591F18091D2028823AC
:1049100009F440C0853009F43FC08091E80083FD70
:104920003DC08091E80082FD2FC08091E80080FFAB
:10493000E9CF2091F3008091F20090E0922B611575
:10494000710559F08830910540F424912093F100CD
:104950003196615071090196F2CF21E0089709F074
:1049600020E08091E8008E778093E800CBCF211182
:10497000CCCF0AC08091D202882361F0853061F0EB
:104980008091E80083FD0AC08091E80082FFF2CFA9
:1049900080E0089582E0089583E0089581E008951D
:1049A000982F973068F59093E900981739F0709137
:1049B000EC002091ED005091F00003C0242F762FE1
:1049C00050E021FD02C09F5FECCF3091EB003E7FB5
:1049D0003093EB003091ED003D7F3093ED0030914E
:1049E000EB0031603093EB007093EC002093ED000E
:1049F0005093F0002091EE0027FDE5CF80E0089570
:104A00008F708093E90081E008958091D30287FF41
:104A100011C08091E80082FD05C08091D202811111
:104A2000F8CF11C08091E8008B770BC08091D20243
:104A3000882349F08091E80080FFF8CF8091E8005A
:104A40008E778093E80008952091E4003091E5008E
:104A500095E64091EC00842F817040FF23C0809147
:104A6000E80080FD1DC08091D202882399F0853036
:104A700099F08091EB0085FD11C04091E4005091C8
:104A8000E5002417350729F3915011F09A01E1CF81
:104A900084E0089582E0089583E0089581E0089518
:104AA00080E008954091E80042FFDDCF08950E9424
:104AB000C5250E94CD25E0EEF0E0808181608083F5
:104AC000E8EDF0E080818F77808319BCA7EDB0E03E
:104AD0008C918E7F8C9380818F7E80831092D10207
:104AE00008950F931F93CF93DF930E94C5250E94D3
:104AF000CD25C8EDD0E088818F7788838881806854
:104B0000888388818F7D888319BC1092D20210928D
:104B1000CE021092D0021092CF0200EE10E0F80107
:104B200080818B7F808388818160888342E060E020
:104B300080E00E94D024E1EEF0E080818E7F8083CF
:104B4000E2EEF0E0808181608083808188608083F4
:104B5000F80180818E7F8083888180618883DF91E6
:104B6000CF911F910F910895E8EDF0E080818F7E45
:104B70008083E7EDF0E080818160808384E082BF04
:104B800081E08093D1020C947125E8EDF0E0808102
:104B90008E7F80831092E20008951092DA001092C6
:104BA000E10008951F920F920FB60F9211242F93D8
:104BB0003F934F935F936F937F938F939F93AF93A5
:104BC000BF93EF93FF938091E10082FF0BC0809130
:104BD000E20082FF07C08091E1008B7F8093E100BB
:104BE0000E9448288091DA0080FF1FC08091D80081
:104BF00080FF1BC08091DA008E7F8093DA00809165
:104C0000D90080FF0DC080E189BD82E189BD09B472
:104C100000FEFDCF81E08093D2020E941A2205C0DF
:104C200019BC1092D2020E9428228091E10080FFDC
:104C300019C08091E20080FF15C08091E2008E7F54
:104C40008093E2008091E20080618093E200809195
:104C5000D80080628093D80019BC85E08093D2028E
:104C60000E942D228091E10084FF30C08091E200FB
:104C700084FF2CC080E189BD82E189BD09B400FEBA
:104C8000FDCF8091D8008F7D8093D8008091E10086
:104C90008F7E8093E1008091E2008F7E8093E2001E
:104CA0008091E20081608093E2008091CE028823AF
:104CB00011F084E007C08091E30087FD02C081E02D
:104CC00001C083E08093D2020E9435228091E100EE
:104CD00083FF29C08091E20083FF25C08091E1001D
:104CE000877F8093E10082E08093D2021092CE020F
:104CF0008091E1008E7F8093E1008091E2008E7FC1
:104D00008093E2008091E20080618093E20042E0C3
:104D100060E080E00E94D0248091F0008860809361
:104D2000F0000E942B22FF91EF91BF91AF919F91D4
:104D30008F917F916F915F914F913F912F910F9044
:104D40000FBE0F901F9018951F920F920FB60F92E3
:104D500011242F933F934F935F936F937F938F9380
:104D60009F93AF93BF93CF93DF93EF93FF93C09144
:104D7000E900CF708091EC00D82FD17080FDD0E891
:104D80001092E9008091F000877F8093F000789482
:104D90000E94E8261092E9008091F00088608093DC
:104DA000F000CD2BCF70C093E900FF91EF91DF9120
:104DB000CF91BF91AF919F918F917F916F915F91B3
:104DC0004F913F912F910F900FBE0F901F9018950C
:104DD0001F93CF93DF93CDB7DEB7AA970FB6F894A2
:104DE000DEBF0FBECDBFE3EDF2E08091F100819315
:104DF00022E0EB3DF207C9F70E9453228091E800C0
:104E000083FF2EC18091D3029091D402492F50E0AC
:104E10004A30510508F024C1FA01EE59FF4F0C94B5
:104E2000BC28803821F0823809F01AC108C080916E
:104E3000CF029091D002992389F082600FC08091B7
:104E4000D7028F70873008F00BC18093E900809102
:104E5000EB0085FB882780F91092E9009091E8002B
:104E6000977F9093E8008093F1001092F100D1C0F9
:104E7000282F2D7F09F0F4C0882319F0823061F0CB
:104E8000EFC08091D502813009F0EAC0933009F07B
:104E900080E08093D0022EC08091D50281112AC07B
:104EA0008091D7028F702FEF280F263008F0D8C0DE
:104EB0008093E9002091EB0020FF1CC0933021F487
:104EC0008091EB00806214C09091EB009061909310
:104ED000EB0021E030E0A90102C0440F551F8A9584
:104EE000E2F74093EA001092EA008091EB008860BC
:104EF0008093EB001092E9008091E800877F809317
:104F0000E8000E940525ACC08111AAC01091D5020D
:104F10001F778091E3008078812B8093E30080915C
:104F2000E800877F8093E8000E9405258091E800D3
:104F300080FFFCCF8091E30080688093E300111133
:104F400002C082E001C083E08093D20289C0805811
:104F5000823008F085C08091D5029091D6028C3DB8
:104F600053E0950779F583E08A838AE289834FB716
:104F7000F894DE01139620E03EE051E2E32FF0E0EA
:104F800050935700E49120FF03C0E295EF703F5F1C
:104F9000EF708E2F90E0EA3010F0C79601C0C096F7
:104FA0008D939D932F5F243149F74FBF8091E80087
:104FB000877F8093E8006AE270E0CE0101960E944C
:104FC000112416C06091D7027091D802AE014F5FD4
:104FD0005F4F0E945523BC01892B09F441C0909179
:104FE000E800977F9093E80089819A810E946F245E
:104FF0008091E8008B778093E80032C0803881F59B
:105000008091E800877F8093E8008091CE028093B2
:10501000F1008091E8008E7772CF811121C08091DC
:10502000D5029091D60299270297D4F48091E80096
:10503000877F8093E8008091D5028093CE020E9402
:1050400005258091CE02811106C08091E30087FD85
:1050500002C081E001C084E08093D2020E943F221E
:105060008091E80083FF0AC08091E800877F8093E9
:10507000E8008091EB0080628093EB00AA960FB667
:10508000F894DEBF0FBECDBFDF91CF911F91089581
:105090000895CF938091D2028823A1F0C091E900B6
:1050A000CF709091EC00892F817090FD80E8C82B23
:1050B0001092E9008091E80083FD0E94E826CF70FD
:1050C000C093E900CF91089587FB082E062687FD3F
:1050D000819567FD61950E94F3280EF4919507FC78
:1050E00081950895AA1BBB1B51E107C0AA1FBB1FD6
:1050F000A617B70710F0A61BB70B881F991F5A9564
:10510000A9F780959095BC01CD01089597FB072ED6
:1051100016F4009407D077FD09D00E94722807FC8E
:1051200005D03EF4909581959F4F089570956195B7
:105130007F4F0895A1E21A2EAA1BBB1BFD010DC0D3
:10514000AA1FBB1FEE1FFF1FA217B307E407F50737
:1051500020F0A21BB30BE40BF50B661F771F881F13
:10516000991F1A9469F760957095809590959B01A9
:10517000AC01BD01CF010895EE0FFF1F0590F49122
:10518000E02D09940E94CA28332312F48A1B9B0B3A
:105190000C94DB28A29FB001B39FC001A39F700DA8
:1051A000811D1124911DB29F700D811D1124911D2F
:1051B00008950E94CA28B7FF0895821B930B089593
:1051C0000E94CA28A59F900DB49F900DA49F800DAA
:1051D000911D11240895B7FF0C94E0280E94E02847
:1051E000821B930B0895991B79E004C0991F9617B1
:1051F00008F0961B881F7A95C9F780950895FC01E1
:105200004150504030F001900616D1F73197CF0150
:105210000895882799270895FB01DC0104C08D912A
:105220000190801921F441505040C8F7881B990B18
:105230000895F999FECF92BD81BDF89A992780B55E
:105240000895A6E1B0E044E050E00C945329A8E1B1
:10525000B0E042E050E00C945329262FF999FECF9C
:1052600092BD81BDF89A019700B4021639F01FBAB9
:1052700020BD0FB6F894FA9AF99A0FBE08950396D6
:10528000272F0E942E290E942D29252F0E942E298A
:10529000242F0C942E290196272F0E942E290C943E
:1052A0002D29DC01CB01FC01F999FECF06C0F2BD2E
:1052B000E1BDF89A319600B40D9241505040B8F7D4
:0652C0000895F894FFCFF1
:1052C600C8003502280850011E0A14010101020017
:1052D6000300030301191A1B1C1D1E1F2021228314
:1052E60021A621872116221222862101E200E90049
:1052F600EA00B500B600B700CD008301CC008A01F4
:105306009201940121022302240225022602270289
:105316002A02B300B4006F007000818283E200E9C4
:1053260000EA00B500B600B700CD008301CC008AC4
:10533600019201940121022302240225022602275A
:10534600022A02B300B4006F007000818283F4F178
:10535600F0956766000102020202060606090909BF
:105366000909090F0F0F0F0F0F1515151819191920
:1053760019191919191919232400FF010001000030
:0A538600FFFF0000010001FF00001E
:00000001FF
